:020000040800F2
:106000002D482C49384A01602C4941602C49816057
:106010002C49C1602C4901612C4941612C498161A5
:106020002C49C1612C4901622C4941622C49816291
:106030002C49C16200F180012C4BCA6143632C4B97
:1060400083632C4B03632C4BC3632C4B03642C4B9B
:1060500043642C4B83642C4BC3642C4B03652C4B47
:1060600043652C4BC3662C4B83652C4B03662C4B32
:10607000C3652C4B43662C4B83662C4B03672C4B20
:1060800043672C4B83672C4BC3672C4808602C4814
:1060900008612C4848602C4848612C48C1E902023C
:1060A0002B488861704710B500F06AFB00F01DFCBA
:1060B000002010BD297500085C0400203F76000810
:1060C00041720008DD7600086191000847770008FA
:1060D000697700088D770008D1A000088572000854
:1060E000EB7A0008E5A400080764000821620008B4
:1060F00069650008CF7C00089D7100087D6B000871
:1061000011920008537100084D640008FF640008F4
:10611000DF8B0008EF710008CD6E0008C565000830
:10612000DB650008ADA300081F6E0008C38F0008E0
:10613000E57C0008097400082394000849A00008C1
:1061400071930008C1A000084571000879A00008FB
:1061500095910008202802D94FF0FF307047B64AC9
:10616000102802EB400204D932F8220D61F31F20FF
:1061700004E032F8020D00F47F4008431080002054
:106180007047AD4A00204FF6FF7122F81010401CF6
:10619000C0B20F28F9D97047F0B50C46A74908449A
:1061A000A1F1240710F8013C581DC6B20A2594FB42
:1061B000F5F005FB104094FBF5F4C0B2202B01D89C
:1061C000B34202D94FF0FF30F0BD395C18465B1C7A
:1061D000DBB2FFF7BFFF002CE9DC0020F0BD9749E0
:1061E000A0F141023E390144192A02D811F8410CAC
:1061F0007047A0F16102192A02D811F8610C7047AA
:10620000A0F13001092901D8C8B270472D2803D068
:106210002E2803D02320704721207047222070476A
:10622000F0B5864E00240D460346243E834F16E00B
:10623000FFF7D5FF315CF81810F8010CFFF78AFF63
:106240005B1CDBB2202B02D94FF0FF30F0BD052CD8
:1062500001D00B2C01D19B1CDBB2641CE4B2285D85
:106260000028E5D1F0BD70B5044673480D462030D6
:10627000FDF7D8FC2846FDF7F9FC7049C0B29A3901
:10628000012388704D7900222DB12044401EC87032
:106290004A700B7103E0CC70401E48700A714A715D
:1062A0008A71CB710B7070BD2DE9F0470346FFF783
:1062B00068FFDFF888A1DFF88891AAF1240AA3B368
:1062C0004FF00008002524E000241AE05B4F5346FD
:1062D0001AF80510385DFFF73DFF3E19595D307C17
:1062E000FFF738FFC82003F0AFFE385DFF21FFF74E
:1062F00031FF307CFF21FFF72DFF641CE4B20F2C2F
:1063000003D899F800000028E0D06D1CEDB21E2DD6
:1063100003D899F800100029D6D008F1010000F048
:10632000FF08B8F10F0FCDD927E0FFE7002556464B
:106330004FF4C8784F46002418E00023315D18461A
:10634000FFF708FF5B1CDBB21E2BF7D9404603F0BA
:106350007BFE0023FF211846FFF7FCFE5B1CDBB22F
:106360001E2BF7D9641CE4B21D2C02D83878002803
:10637000E3D06D1CEDB2282DDDD999F8000010B9DD
:10638000304901200860FFF7FCFE2C4901207D39CF
:10639000FFF746FFBDE8F0472849613909203FE78C
:1063A000254810B5182228492030FDF78AFC2349DA
:1063B00000209A390870BDE81040E2E6F0B51E4DA5
:1063C0001E4E00232035243E06F14407A6F1760434
:1063D00010E0102B03D9C3F11800285C00E0E85C42
:1063E000FFF7FDFE315C2078C01A385CFFF7B2FE83
:1063F0005B1CDBB220788342EBD9C0B2401C20701A
:10640000F0BD7047704710B50B4C0021203400F0F0
:106410000F02C1F105030009E254092A01D94132F2
:1064200000E03032491CC9B2E2540629EFD3002003
:10643000A0710148203010BD740900200A0300201B
:106440004008002044080020470A002070B57C4D19
:10645000420716D50C0901F00F01820702D5285D0D
:10646000484005E0C00705D0285DC1F10F01084094
:10647000285500E02955734E30887349C00724D150
:1064800020E0242902D94FF0FF3070BD4A1ED317F7
:1064900002EB9372C2F3870422F00302491E8A1AA8
:1064A00001219140C9B2C20702D0285D084305E02E
:1064B0008007285D01D5484000E08843285500F05A
:1064C0000F00D5E70888C00708D03088C007FCD186
:1064D0000888C007F9D1052003F0CEFD5B48C168EC
:1064E0002A5D01F46F41D243120741EA1261214350
:1064F000C16001213046FAF789FE002070BD2DE908
:10650000F05F00244F4EDFF838A14FF0030BDFF8A7
:106510004081F025DFF830914C4F1AE0CCB1042CCB
:106520001DD0002132883046D207FBD1B9F80020B7
:10653000D207F7D1FA6802F46F4222430A43FA60A5
:106540000121FAF763FE641CE4B2092CE6D3BDE82E
:10655000F09F9AF800102BEA01000101E2E798F899
:10656000000025EA0001DDE72DE9F05F0024344D4D
:10657000344E4FF0030A4FF0C00BA046DFF8C8902E
:10658000324F19E0C4B1F02105F80480328830465A
:10659000D207FBD1B9F80020D207F7D1FA6802F48C
:1065A0006F4222430A43FA600121FAF72FFE641C6E
:1065B000E4B2092CE6D3CAE729782AEA01004BEABB
:1065C0000011E3E71E49002001F10A020B5C13549D
:1065D000401CC0B20928F9D3704770B5184D00248B
:1065E0000A35285D40EA0410C1B20420FFF72EFFEF
:1065F000641CE4B2092CF4D370BD70B5154C4FF493
:1066000096704FF4FA76144D20600FE0FFF777FF95
:10661000304603F019FDFFF7A7FF287810B9304680
:1066200003F012FD2168491E216002D0287800285D
:10663000ECD02878002801D10120206070BD000036
:10664000AD09002000040040000800400010014097
:106650007D050020440800204008002070B5F54D5D
:106660000420F549287102200870F44800240470C1
:10667000F348047003F0B1F8F349F2480860F349B5
:106680000860F3486C70EC70047070BD10B5E94C94
:10669000012060712178C0B2FFF75CFD6079401C79
:1066A000C0B260712028F5D9207810B14000207068
:1066B00010BDFF20FBE7FEB5E64801241D2607C8F4
:1066C0008DE8070000272546684603F06FFE01E0CD
:1066D000112C06D02146641CE4B20120FFF7B6FE5F
:1066E00000E012243146761CF6B20020FFF7AEFE21
:1066F000642003F0A9FC242C00D10124242E00D115
:1067000001267F1CFFB20A2F09D129466D1CEDB26C
:10671000002000F033FA092D00D10125002700F0F8
:1067200094FB0028D4D000F0B5FB0028D0D19DF810
:10673000000003F0D7FEFFF724FDC7A10120FFF7FB
:106740006FFDC9A10D20FFF76BFD0020FEBDC04904
:1067500010B501200870C84964200860C749086066
:10676000C749C84802F086FBC7A10120FFF758FDC2
:1067700003F0ABF9FCF713FBBDE81040FFF701BDD8
:1067800070B5C348016841F4E0210160C1494FF48C
:106790007A700860C049DC200870C0490F2008707A
:1067A000FCF759FBFCF7D3FBFCF7A0FBFAF7FEF96B
:1067B000FCF71BFDFCF734FBFCF732FCFCF75FFC3D
:1067C000FCF788FCFCF708FCFFF71AFCB44800252E
:1067D000C0F8B4510121C0F8B011FCF726FBFDF759
:1067E00020FD30B9FDF777FB0120FDF7B4FCFDF784
:1067F00078FBAC480570FFF7C4FC00F0FEF9FFF72A
:10680000B3FE00F02CFBFCF7D8FD03F0ECFC03F02A
:1068100046FCFFF723FF0020FCF7AAFAFCF72FFC49
:10682000FCF758FC8A480078401E102802D300204C
:10683000FFF78DFFFCF709FA0020FCF7A4FA9A4C49
:106840009A4E2168884201D1307880B398A1012006
:10685000FFF7E6FC98A10920FFF7E2FC02F03CFFFD
:1068600035700020FCF78FFA20600020FCF760FAFA
:106870004FF4487003F000FC0020FCF784FA216814
:10688000884212D08EA10120FFF7CAFC8EA10920F8
:10689000FFF7C6FC4FF4C87003F0EEFBFCF78DFD6C
:1068A000642003F0E9FBFCF788FDFFF76AFCFFF7C3
:1068B0005BFE87A10120FFF7B3FC87490B20FFF7A0
:1068C000AFFC86A11120FFF7ABFC864801681B20B6
:1068D000FFF7A6FC4FF4FA7003F0CEFB8248006885
:1068E000804702F006FB002070BD804F564EDFF857
:1068F0004891DFF8FCB1DFF8FCA14FF000084D4CE7
:106900002079012801D0022819D1E078032814D178
:1069100079487A4900680978007A88420DD0784928
:10692000FCF712FD77A17C48FDF77CF974497A48A1
:10693000FDF7BBF97848FDF7F2F803F070FD434D21
:106940003168286888424CD000F0A4FAA070E17841
:1069500089B1FF280FD000F089FA6949FCF7F4FCEF
:106960006EA16D48FDF75EF965496B48FDF79DF92D
:106970006948FDF7D4F899F800000228A07809D0FA
:10698000FF281ED0C0B2152807D0052808D802F06D
:106990008AFE12E00328F5D913E002F05CFD0CE05A
:1069A00000F064FA624909688847002805DAE0784F
:1069B000012802D15FA0FDF7B2F88BF800808AF8B9
:1069C0000080387850B96548007803F055FB286896
:1069D0003168884202D0A07800F078FA87F8008009
:1069E000AEE799F80000012813D19BF800102D297B
:1069F0000BD38BF80080E078012802D958A0FDF76E
:106A00008EF85D480068804703E09AF800108BF824
:106A100000109AF80000544648B1224D2878012809
:106A200005D1FCF7F9FF85F8008084F8008001F0BB
:106A3000C5FA64E7AE03002093050020850300201B
:106A400040080020270A0020500500204C050020A7
:106A50002404002050A50008202020206E697775AE
:106A60006D7066200000000020202041524D7072A1
:106A70006F6A656300000000300400202C040020D1
:106A80001007002009070020202067616D650000C5
:106A900024ED00E0F8030020C0030020CF03002015
:106AA000000022421E0000203C040020CB030020F6
:106AB00020726573657400006E7672616D2000004F
:106AC000206E7672616D000073686F742020000084
:106AD00020702D72657600004106002020672D721F
:106AE00065760000340700203C0700207605002072
:106AF0002908002028080020480800204C06002013
:106B0000C10900204576656E7420747269676765F7
:106B100072202D2000000000970A0020537769742E
:106B2000636820436C6F736564202D2000000000B3
:106B300038070020537769746368206E6F74207083
:106B4000726F6772616D6D656420666F7220746824
:106B500069732067616D653F213F000008070020D1
:106B60005761746368646F672042616C6C20536581
:106B7000617263682E000000F80500202DE9F041E5
:106B80008446082937D88D4A8D481388DB07FCD105
:106B90000388DB07F9D18B4C5FEACC724FF001051B
:106BA000E2680FD04DF6FF731A404A40E2600027BA
:106BB000854E032910D9BCF1020F0DD20121FAF73D
:106BC00025FB14E002F45F434A1E05FA02F2C2F10B
:106BD000FF021343E360EAE7C6F8B451C6F8B471A4
:106BE000282003F049FAE06840F0FF00E060C6F8B2
:106BF000B451C6F8B471BDE8F081724810B5C168EF
:106C000041F0FF01C160704C0120C4F8B40104F5EB
:106C1000DA7403F019FA0020206010BD2DE9FC5F42
:106C20006AA00026D0E90010CDE9001001254FF43C
:106C3000487ADFF8A0814FF47A7BDFF89C91A8E0D6
:106C400066A10720FFF7ECFA01210020FFF7FEFB09
:106C5000C82003F011FA01210846FFF7F7FB02F004
:106C6000ADFE00287BD15446504603F005FA02F0F1
:106C7000A5FE0028F6D15AA10720FFF7D1FA02217C
:106C80000120FFF7E3FBC82003F0F6F90221002002
:106C9000FFF7DCFB02F092FE00287FD1204603F0D4
:106CA000EBF902F08BFE002878D14E48007890B1C5
:106CB0004DA10720FFF7B4FA11210120FFF7C6FB11
:106CC00098F8000003F0D8F911210020FFF7BEFB6F
:106CD000584603F0D1F902F071FE00285ED1434816
:106CE0000078B0B199F80000092812D040A107201F
:106CF000FFF796FA12210120FFF7A8FB98F8000091
:106D000003F0BAF912210020FFF7A0FB584603F068
:106D1000B3F902F053FE10BB36A10720FFF780FA4B
:106D2000002423E06F461DF804100820FFF734FA12
:106D3000395D0020FFF722FF16B14FF4FA6000E042
:106D4000584603F099F900F0B7F8032803D100F092
:106D5000A1F82EB100262EB16D1CEDB204E01DE0AD
:106D60000126F8E7641CE4B2072C04D800F0A4F86C
:106D700008B1142DD6D399F80000092803D11221A7
:106D80000020FFF763FB00F06AF86D1CEDB2142DD4
:106D900004D802F013FE00283FF452AF02F00EFEBA
:106DA00010B915490120086001210020FFF74EFBB2
:106DB00010A10720FFF734FABDE8FC9F0004004053
:106DC00000080040001001400000224204050102BA
:106DD00003060708C0030020240400204C310000F3
:106DE0004C320000790500204C3300007A05002069
:106DF0004C34000020200000440800200A21B0FB91
:106E0000F1F201FB1202B0FBF1F1C24B012088400C
:106E10009A5C024201D0002070470120704730B5D3
:106E2000BC4CBD4B0C3C2246A16852684FF0FF356C
:106E3000994201D11F3B00E04B1C9A4201D12846E8
:106E400030BD08700020A36030BDB2480C38D0E9D6
:106E50000110814201D00120704700207047AE48E8
:106E6000AC491F380C3988604860704700F00F014A
:106E7000000900EB800001EB4000C0B270470A211E
:106E8000B0FBF1F201FB1202B0FBF1F002EB0010DB
:106E9000C0B270479F4A0C3AD2E90110814201D139
:106EA000FF2070479C4B0878994202D1A3F11F0143
:106EB00000E0491C5160704796490C39D1E9010145
:106EC000884201D1FF2070470078704730B5914C5F
:106ED000914A0C3CFF23616809E00D78854200D19E
:106EE0000B70914202D18C491F3900E0491CA56802
:106EF000A942F2D130BD70B5884C0546207840B12A
:106F0000874E3078012804D1FCF786FD00203070D0
:106F10002070804C0C3CD4E90101884209D12846FC
:106F200003F092F8D4E90101884202D14FF0FF301A
:106F300070BDBDE87040ADE770B500254FF4167622
:106F40003046FFF7D8FFC4B2032C06D02CB16D1C1D
:106F5000EDB23C2DF4D3002070BD4FF4C870FFF7A4
:106F6000CAFF40B1032802D0032C0AD005E0032C4D
:106F700007D024B101E0032C01D0032070BD022012
:106F800070BD012070BD2DE9F041624E00254FF427
:106F900096773846FFF7AFFF040002D5F078C007B8
:106FA00008D0032C07D034B16D1CC82DF1DB0020B4
:106FB000BDE8F08103244FF4C870FFF79CFF40B197
:106FC000032802D0032C0AD005E0032C07D024B1FB
:106FD00001E0032C01D00320EAE70220E8E70120CA
:106FE000E6E710B5FFF7A8FF4E49087010BD10B5D1
:106FF000FFF7C9FF4B49087010BD464A0A210C3AF9
:107000001078B0FBF1F301FB1301052901D0401CFE
:1070100002E04B2802D0401D107070470020FBE7B3
:107020002DE9F0413B4E00250C3EDFF8FC803F4F40
:1070300064E04FF44870FFF75EFF040008D0032CB3
:1070400001D055B921E00DB1002557E0012555E0EB
:107050000020386052E0FFF7D0FF3078FFF7CEFE17
:1070600010B930780028F6D131A11520FFF7D8F8F3
:10707000317829B11620FFF78FF8FFF7BEFF3DE00A
:10708000012131702AA116202DE0002C2EDDE0B266
:10709000FFF7ECFE01461620FFF77EF81420FFF7FD
:1070A0002AFFA0422AD103210020FFF767FD012417
:1070B00020A10120FFF7B4F841460920FFF7B0F8FE
:1070C000FA2002F0D9FFFFF75CF8642002F0D4FF49
:1070D000641C042CECDDFFF7C2FE18490120FFF709
:1070E0009FF841460920FFF79BF807E010A1152003
:1070F000FFF796F800211620FFF74EF83868401E7B
:107100003860401C95D1BDE8F0410DA11520FFF776
:1071100087B8000054050020460A002028080020F7
:107120001E00002075050020BE020020440800203B
:1071300020000000636C65616E2000008D0200205D
:107140002020000010B5FFF759FE002800D00120D4
:1071500010BD10B5FC4C60790A280AD3142801D35D
:10716000A07800E0607884F82200C1B20120FFF727
:107170006DF960790A21B0FBF1F201FB1200E064C5
:1071800000280AD021780844401EC1B284F8221099
:10719000BDE810400120FFF759B910BD10B5EA4C09
:1071A0006079142806D01D2804D00A2804D013289A
:1071B00002D007E0A17812E0617884F82210002064
:1071C000FFF744F960790A21B0FBF1F201FB1200EC
:1071D000E06400280AD021780844401EC1B284F837
:1071E0002210BDE810400020FFF730B910BD10B5E7
:1071F000D54C607994F82310884207D2FFF7CEFF70
:107200006079401C6071BDE81040A2E710BDCF4A14
:10721000CF4811780078814201D300280FD1491C52
:10722000C9B2117018B90F2901D90F201070C948BF
:107230000078002803D011781020FEF7ADBF70470A
:1072400010B504210020FFF799FCC34800780028FE
:1072500017D1C248BD4A0168491C0160BC48117879
:107260000078814201D300280BD1491CB948C9B22A
:1072700011700078002804D0BDE810401020FEF7FF
:107280008BBF10BD10B5B648AF4C007818B1217B4C
:10729000206C884208D0B348007810B1FFF7D0FFC7
:1072A0000AE000F041F907E0AF48006800F0ACF8F0
:1072B00004210020FFF762FC207B206410BD024601
:1072C000AA48016800290FDD8A420BDDA848006842
:1072D000884209DD824206DDA6490968814203DD54
:1072E0008A4201DA084670470020704710B5A24A6A
:1072F000954C1168607C491C012810D0022819D0D7
:10730000032822D0E36E002B2ADDA06E984227DDF1
:107310001160FFF7D4FFE066BDE81040B2E7636D8F
:10732000002B1DDD206D98421ADD1160FFF7C7FFAD
:107330006065F1E7E36D002B12DDA06D98420FDD73
:107340001160FFF7BCFFE065E6E7636E002B07DD29
:10735000206E984204DD1160FFF7B1FF6066DBE745
:1073600010BD794B10B518465A7C816F007A012AFE
:1073700008D0022A0CD0032A10D09A6E11449966C4
:1073800090B114E01A6D1144196580B906200CE023
:107390009A6D1144996550B90E2006E01A6E114499
:1073A000196620B9162000E01E20FEF7F5FEBDE8A4
:1073B00010409BE764488030406C004710B5624C39
:1073C000E07A00281FD10120E072A07B18B90421C7
:1073D0000020FFF73BF869480078002813D094F8A4
:1073E000330010B194F8340002E094F8341021B165
:1073F00018B955488030406C804761480078BDE836
:10740000104003F06FB810BD2DE9F0410446FFF7BE
:10741000D5FF4D4DA87A002870D1012085F837009E
:1074200005F18000806B804756484FF47A76564FBE
:107430000068E863B44233DB42F22830844216DC51
:1074400094FBF6F006FB1040E8BB94FBF6F43878AA
:1074500018B103210020FFF791FBAE67FFF781FF12
:10746000641E002C5EDDE86B02F006FEEFE742F2E0
:10747000107694FBF6F006FB104020BB94FBF6F46C
:10748000387818B105210320FFF778FBAE67FFF7C6
:1074900068FF641E002C45DDE86B02F0EDFDEFE7B0
:1074A000642C1DDBB4F5617F3CDC642094FBF0F1BF
:1074B00000FB114139B994FBF0F46426387828B107
:1074C0000221002000E015E0FFF758FBAE67FFF750
:1074D00048FF641E002C25DDE86B02F0CDFDEDE7D2
:1074E0000A2C07DB5A2C1DDC0A2094FBF0F100FB70
:1074F000114121B1AC67BDE8F04132E712E094FBE5
:10750000F0F40A26387818B101210020FFF736FB85
:10751000AE67FFF726FF641E002C03DDE86B02F068
:10752000ABFDEFE7BDE8F08110B51848064C0078D8
:10753000A17B884237D90848007820B10A48006802
:10754000BDE8104060E723E05C050020D203002086
:10755000D0030020C7030020D5030020F003002043
:10756000C1030020C203002018040020FC030020F7
:10757000100400201C04002008040020CE0300207A
:10758000D006002030040020CD030020D1030020CD
:1075900004210120FEF75AFFA07B401CA073FE4887
:1075A0000168491C016010BD30B5FD49FB48A1F1DF
:1075B00080040A690068217CFA4B50B1884208D9DE
:1075C0001D68411A6943B1FBF0F1B2FBF0F21144BE
:1075D00001E092FBF1F11960F3490A78002A2DD0FD
:1075E000F2490A28096802D8B1EB500F26D9642560
:1075F0006943B1FBF0F1A167881A1B6864305843F6
:1076000090FBF5F042F2107390FBF3F05843E84B17
:10761000984200DDE748914210D0E74900EB0012A4
:10762000E64B08600A2192FBF1F21A6000EBC002FF
:1076300002EB001090FBF1F0E149086030BD70B53D
:10764000D74C803CA07994F82810884211D204F1DC
:10765000CC05284410F8011C11B10020FEF7F6FEFD
:10766000A079295C11B10120FEF7F0FEA079401C41
:10767000A07170BD70B5CA4D803DA879012816D99A
:1076800005F1CC04204410F8011C11B10020FEF7D4
:10769000DDFEA879401EC0B2A871204410F8011C7C
:1076A000002904D0BDE870400120FEF7CFBE70BDB8
:1076B000BB488038417F31B190F82210112902D1A6
:1076C000122180F82210817F002906D090F8221024
:1076D000122902D1132180F82210704770B5B04CE6
:1076E000803C2046E17F90F82400052341B12246EA
:1076F00092F820506A1CD2B2814206D1E3770BE0A7
:10770000E377401F84F8200008E0491CE1778542B8
:1077100002D184F8203001E084F8202014F81F0FF3
:10772000E070FFF7C5FFE17821700120FEF78EFEC3
:107730006078E070FFF7BCFFE1786170BDE87040F1
:107740000020FEF783BE9649954880394A7E012A7B
:1077500001D04A6F01E002684A67CA67012110221E
:10776000C0E902214160704710B511210120FEF7E8
:107770006DFE94488A4980390078C86302F07CFC29
:107780001121BDE810400020FEF760BE10B51221A7
:107790000120FEF75BFE8B48814980390078C86381
:1077A00002F06AFC1221BDE810400020FEF74EBE38
:1077B000854810B50078002807D0FFF741FDBDE8E7
:1077C00010404FF4967002F057BC10BD70B5744C69
:1077D000803CE07A0028A06B01D0401EA063012508
:1077E00028B1207970B10020207104210DE0A07B28
:1077F0004FF0040120B10120FEF728FEE57070BDB6
:107800000020F9E7257104210120FEF71FFEBDE8E5
:10781000704063487C3002F0C9BD2DE9F05F604ED6
:107820000024803EDFF8A481DFF87091DFF8A0A18A
:10783000DFF8A0B1684F7476012568A10120FEF73A
:10784000EFFC66A10920FEF7EBFC707D01280ED14C
:1078500064A1FEF7E5FC65A10920FEF7E1FC98F8BC
:1078600000107167717E022901D188F80040707D97
:1078700002280FD15FA10120FEF7D2FC5FA10920F1
:10788000FEF7CEFCD9F800107167717E022901D194
:10789000C9F80040707D03280FD15AA10120FEF7DE
:1078A000BFFC5AA10920FEF7BBFCDAF80010716793
:1078B000717E022901D1CAF80040707D04280FD1E1
:1078C00050A10120FEF7ACFC52A10920FEF7A8FC54
:1078D000DBF800107167717E022901D1CBF80040FE
:1078E000707D05280ED13FA10120FEF799FC4BA128
:1078F0000920FEF795FC4B4801687167717E0229EB
:1079000000D10460707D06280ED147A10120FEF74A
:1079100087FC47A10920FEF783FC4748016871678F
:10792000717E022900D10460707D07280ED13EA12E
:107930000120FEF775FC41A10920FEF771FC1648F5
:1079400001687167717E022900D10460707D08288A
:107950000ED135A10120FEF763FC3AA10920FEF704
:107960005FFC3A4801687167717E022900D10460AA
:10797000707D09280ED136A10120FEF751FC36A1F9
:107980000920FEF74DFC074801687167717E0229E6
:1079900000D10460707D63E0E8030020DC03002078
:1079A000DC0500200C040020B9030020080400209E
:1079B000801A060070F30500FC030020100400206C
:1079C0001C040020C0030020C9030020D2030020B3
:1079D000E0030020E40300204907002020202020AD
:1079E0002020000020746F74616C00006372656475
:1079F00073000000202067616D6500007374617280
:107A00007473000020636F696E730000206C6566FC
:107A10007400000072696768740000007265706C21
:107A200061730000F00300206E756D6265720000E6
:107A3000736C616D73000000EC0300206562616C83
:107A40006C73000074696C7473000000F403002010
:107A5000617665726167000073636F726520000074
:107A6000B17D88420FD1FEA10120FEF7D9FBFEA116
:107A70000920FEF7D5FB4FF0FF307067FC484460EB
:107A8000707E012817D0AFF2AC011120FEF7C8FBC1
:107A9000716F002902DB1620FEF77EFB706C401E22
:107AA0007064FFF7A4FA707E012811D0022811D06B
:107AB000032811D000E07575AFF2E0010920FEF750
:107AC000AFFBAFF2E801BDE8F05F1920FEF7A8BBFD
:107AD0003D70B2E67576FBE7707DB17D884201D1DD
:107AE0007575AAE6401C7075A7E6E14810B58038A8
:107AF0000146447EC97C01220023012C02D019B129
:107B0000C26702E041B1C374C367C16F4167D8481F
:107B1000C0E90223426010BDC274F1E7D548007885
:107B200000280AD0D2490022803900EB4000CA70F8
:107B3000886301F1FC0002F039BC70472DE9F04187
:107B4000CD48CB4D0078803D40B9CC48696F81422B
:107B500004DD91FBF0F200FB12106867C84C686FFF
:107B60002168884225DDC74E307808B1FFF720FE36
:107B7000C54F686F396888421CDD2160C34C21689D
:107B8000884215DD307808B1FFF712FE20683860B2
:107B9000BF4F686F396888420CDDFFF709FE307807
:107BA00018B9FFF705FEFFF703FE38682060686F1D
:107BB0003860B7E42060B5E470B5AD4C0120803C7E
:107BC0006425A064206D606790FBF5F105FB110052
:107BD000E064E17B884201D1FFF732FBA06C401CDE
:107BE000A064217C88420AD8022804D0032804D04B
:107BF000A06E6067E8E7A06DFBE7206EF9E770BD57
:107C00009B4A10B5803A0023516F491E5167906C12
:107C1000C2E9123001230F280AD0082819D90224FA
:107C20000E280BD0002908D100F00700546714E09B
:107C3000002902D103209364506710BD39B992F82E
:107C40003700012802D05467946410BD53679364D1
:107C500010BD0029FCD1401C5367906410BD0F2853
:107C600003D0082803DD022070470320704701205D
:107C7000704710B587487E4C0121803C0068E06366
:107C80000020FEF77BFFE06B02F0F6F901210020F7
:107C9000FEF774FFE06B400002F0EEF901210020D6
:107CA000FEF76CFFE06B400002F0E6F903210020D4
:107CB000FEF764FFE06B02F0DFF902210020FEF71F
:107CC0005DFFDC20E063BDE8104002F0D5B96848F4
:107CD00071498038407C022801D8112000E0012041
:107CE000FEF79EBA10B5624C803C607C0228AFF271
:107CF000143114D81120FEF793FAAFF22031192075
:107D0000FEF78EFA607C022803D91620216EFEF75A
:107D100043FA607C032817D91E20A16E10E00120D1
:107D2000FEF77EFAAFF24C310920FEF779FA062011
:107D3000216DFEF731FA607C012805D9A16D0E2076
:107D4000BDE81040FEF728BA10BD10B553A10120C0
:107D5000FEF766FA5348007808B153A100E054A139
:107D60000920FEF75DFA424C803CE079D8B152A17F
:107D70001120FEF755FAAFF29C311920FEF750FAA8
:107D8000E07990B1012812D04D4801681E20FEF71D
:107D900003FAE079401CC0B20321B0FBF1F201FB11
:107DA0001200E07110BD47A1E2E74848EDE74848FE
:107DB000EBE770B5364E2E4C304D3068803CA84213
:107DC00043DD206FA84214D1AFF2F0313248FBF707
:107DD00029FF31490120FEF723FA2F490920FEF738
:107DE0001FFA2D491120FEF71BFA2B491920FEF727
:107DF00017FA3068216F90FBF1F106206167FEF7FA
:107E0000CBF92048007848B320480168A94203DD37
:107E1000206F91FBF0F161670E20FEF7BDF91A4863
:107E20000168A94203DD206F91FBF0F16167162024
:107E3000FEF7B2F912480168A94203DD206F91FBF9
:107E4000F0F161671E20FEF7A7F9206F012850D0DE
:107E50000A2190FBF1F0206705483BE03FE000007D
:107E6000202064617461000020646F6E6520000052
:107E7000DC050020BA030020C803002040420F00A8
:107E800000040020C503002020040020140400206A
:107E90000404002030040020470A00202065787484
:107EA00072610000C203002067616D652020000040
:107EB00062616C6C20200000616E642061740000BF
:107EC0001C0400202020617420200000FC030020FE
:107ED00010040020BDE87040943002F067BA0E2014
:107EE000616FFEF759F91620616FFEF755F9616F62
:107EF000A8E72567B0E770B5FE4CA07C00285CD0F1
:107F0000FD4D216DA9420CDD206FA84204D1AFF2D6
:107F100034510120FEF784F9216F206D90FBF1F1BF
:107F200061670620FEF738F9A16DA9420CDD206FCC
:107F3000A84204D1AFF25C510920FEF771F9216F1C
:107F4000A06D90FBF1F161670E20FEF725F9216E1F
:107F5000A9420CDD206FA84204D1AFF2805111205C
:107F6000FEF75EF9216F206E90FBF1F1616716203C
:107F7000FEF712F9A16EA9420CDD206FA84204D1D0
:107F8000AFF2A8511920FEF74BF9216FA06E90FBBC
:107F9000F1F161671E20FEF7FFF8206F012808D07D
:107FA0000A2190FBF1F02067D448BDE8704002F050
:107FB000FDB9D24825670C30F7E770BD2DE9F041D7
:107FC000CC4C207F002874D1AFF2F051CC48FBF7A5
:107FD00029FE94F837000025C74F0126022810D04B
:107FE000E17A002965D1042863D0207DA17C084373
:107FF0005FD1E07E00287DD0E576207A00287AD017
:10800000C2E0BC488030006B8047207D002850D102
:10801000BC48007800284CD0B9490120FEF700F98F
:10802000B7490920FEF7FCF8B5491120FEF7F8F82A
:10803000B3491920FEF7F4F8062002F053FA07209E
:1080400002F050FA042002F04DFAE07EDFF8B88228
:10805000D8B1E57603210020FEF7F8F998F8000082
:1080600028B1A07C18B12767FFF745FF55E006202F
:10807000216DFEF791F80E20A16DFEF78DF8162008
:10808000216EFEF789F8A16E44E0A048E6760078FC
:1080900080B1E674E07D401CC0B2E07502280AD9C8
:1080A000E571FFF752FE9548183802F07FF9E57543
:1080B00033E070E0E57403210120FEF7C7F998F87A
:1080C0000000934D30B12868B84203DD2767FFF701
:1080D00070FE22E006202968FEF75EF88D480078E1
:1080E00078B18D4801680E20FEF756F88B4801687C
:1080F000162001E02DE014E0FEF74EF888480168F4
:1081000008E00E202968FEF747F816202968FEF7D8
:1081100043F829681E20FEF73FF87848267530306E
:1081200035E0607C012806D0022807D0032808D05B
:10813000042809D028E07249012007E0704909208D
:1081400004E06F49112001E06D491920FEF768F83D
:108150001AE02767207AB0B9607C012806D002288F
:1081600007D0032808D0042809D00CE00620216D90
:1081700007E00E20A16D04E01620216E01E01E2014
:10818000A16EFEF709F8E6765C4826753C30BDE83E
:10819000F04102F00BB90CE5564901F180004A7E2E
:1081A000012A01D04A6F01E002684A67CA675D4947
:1081B000C1605D49816042F21071416070472DE9F4
:1081C000F05F4C4E002501277576DFF84C91DFF803
:1081D0004CA1DFF83C81DFF848B186F8257006F144
:1081E0008004AFF608010920FEF71AF896F825007A
:1081F000012811D1AFF2D071FEF712F84BA109207E
:10820000FEF70EF84B4B18787067FFF79CFA96F85C
:10821000740018700820A06096F8250002280ED17E
:1082200045A10120FDF7FCFF45A10920FDF7F8FF5E
:10823000454B18687067FFF7AFFF706F186096F8CE
:10824000250003280ED141A10120FDF7E9FF3CA143
:108250000920FDF7E5FF3F4B18687067FFF79CFFAB
:10826000706F186096F8250004280ED13AA10120FD
:10827000FDF7D6FF32A10920FDF7D2FF384B186871
:108280007067FFF789FF706F186096F82500052862
:1082900010D134A10120FDF7C3FFAFF6440109203E
:1082A000FDF7BEFFD8F8000043467067FFF774FF84
:1082B000706F186096F82500062812D12BA10120B6
:1082C000FDF7AEFF2BA10920FDF7AAFF0F4B187891
:1082D0007067FFF738FA96F8740018701E20C4E92A
:1082E000020596F8250007285BD124A10120FDF79F
:1082F00097FF47E05C05002040420F007C0600200D
:10830000470A0020C6030020C8030020B90300204C
:1083100004040020C50300201404002020040020D1
:108320000004002080380100301B0F0062616C6C7B
:1083300073000000BB0300202066697273740000A4
:108340007468726573680000FC0300207365636FD6
:108350006E640000100400202074686972640000DC
:108360001C040020202068696768000020206175D7
:10837000746F000070657263656E0000202062619A
:108380006C6C0000FEA10920FDF74AFFFE4B187837
:108390007067FFF7D8F996F8740018702820C4E9C0
:1083A000020596F82500082811D1F8A10120FDF753
:1083B00037FFF8A10920FDF733FFDFF8E0C39CF891
:1083C0000000F074FFF791FBF07C8CF8000096F849
:1083D0002500092811D1F2A10120FDF721FFF2A10A
:1083E0000920FDF71DFFDFF8C8C39CF80000F074FA
:1083F000FFF77BFBF07C8CF8000096F825000A283C
:1084000028D1E2A10120FDF70BFFEAA10920FDF729
:1084100007FFDFF8A8C39CF80000F074FFF765FBC6
:108420009CF80000012812D1F07C80B9E44AD8F809
:10843000001091420BDDE349C8F80010E249C9F889
:108440000010E249CAF80010E149CBF80010F07CB6
:108450008CF8000096F825000B2813D1AFF67C218C
:108460000120FDF7DDFEDBA10920FDF7D9FEDB4B86
:1084700018787067FFF767F996F874001870052090
:10848000C4E9020596F825000C2811D1D4A10120D9
:10849000FDF7C6FED4A10920FDF7C2FEDFF850C3E8
:1084A0009CF80000F074FFF720FBF07C8CF80000D3
:1084B00096F825000D2811D1CEA10120FDF7B0FEC0
:1084C000CEA10920FDF7ACFEDFF838C39CF8000010
:1084D000F074FFF70AFBF07C8CF8000096F825009A
:1084E0000E2811D1C8A10120FDF79AFEC8A10920CC
:1084F000FDF796FEDFF820C39CF80000F074FFF74C
:10850000F4FAF07C8CF8000096F825000F2811D1C1
:10851000C2A10120FDF784FEC2A10920FDF780FE63
:10852000DFF808C39CF80000F074FFF7DEFAF07C77
:108530008CF8000096F8250096F82710884205D39D
:1085400096F82610884201D2606B804796F8250085
:1085500096F8261088420ED1B5A10120FDF760FEE5
:10856000B5A10920FDF75CFE4FF0FF307067656034
:10857000707E012818D0AFF69C311120FDF750FE17
:10858000716F002902DB1620FDF706FE706C401E9D
:1085900070640BD0FEF72BFD707E012811D00228ED
:1085A00044D0032846D001E086F82570A0A1012020
:1085B000FDF736FEAFF6DC31BDE8F05F0920FDF7D0
:1085C0002FBED4E90110421AF06F824201DAE0684E
:1085D00000E00844206096F82500052823D1206893
:1085E00090FBF1F0484344F62061C8F8000088424F
:1085F00003DD421AC9F8002001E0C9F8005047F233
:108600003051884203DD411ACAF8001001E0CAF86F
:10861000005049F64041884203DD401ACBF8000083
:1086200001E0CBF8005086480770DAE5E06820608A
:108630007776F8E796F8250096F82610884202D15A
:1086400086F82570CDE5401C86F82500C9E510B5F3
:108650007C487D4C03210068E0630020FEF78EFA21
:10866000E06B01F009FD02210020FEF787FAE06BC4
:1086700001F002FD01210020FEF780FAE06B01F01D
:10868000FBFC02210020FEF779FAE06B01F0F4FC1C
:10869000E06B01F0F1FC01210020FEF76FFAE06BC6
:1086A00001F0EAFC03210020FEF768FABDE8104063
:1086B000012001F017BF654B654800211980026851
:1086C000002A15D06048406F904211DD614A491C74
:1086D00019801268002A0BD0904209DD5E4A491CBD
:1086E00019801268002A03D0904201DD491C1980CC
:1086F00070475549886C0F2803D0082803D90220F9
:1087000002E0032000E0012088647047704753486E
:1087100010B501684C4C491C016051480078A064B8
:1087200094F82A006067FFF76BFA94F8740084F8F5
:108730002A004C48007808B1FFF79BFAA06C00288B
:1087400005D0FEF764FDA06C401EA064F7E710BDE5
:108750002DE9F0473C4E0025DFF80C91DFF8E0A052
:1087600075764FF00F0806F180040127AFF694519B
:108770000920FDF755FD96F82D00012876D176E009
:108780007361766520200000BA030020656E616287
:108790006C6500003420485354440000C503002099
:1087A000202073686F7700006873746420200000D5
:1087B000C60300206D696C696F6E0000C80300205D
:1087C00040420F00E0E60B0020120A00603D080066
:1087D000A068060074696C7473200000D303002045
:1087E0002069646C65200000616E696D6174000031
:1087F000CA0300202066617374200000626F6E75EA
:1088000073200000C303002020736B696C6C0000B0
:1088100073686F7420200000CE0300205475726EC0
:108820006D7400004D6F646520200000D5030020AA
:108830002073657475700000646F6E652020000001
:1088400049070020300400205C050020B40300200C
:10885000FC030020100400201C040020E003002082
:10886000BD030020CC0300201804002014E0FEA16A
:10887000FDF7D6FCFEA10920FDF7D2FCFE4B1878CF
:108880007067FEF760FF96F874001870FFF7E7F95D
:1088900086F82A00C4E9028596F82D00022815D131
:1088A000F6A10120FDF7BCFCF1A10920FDF7B8FC01
:1088B000F44B18787067FEF746FF96F8740018704E
:1088C000FFF7CDF986F82B00C4E9028596F82D0054
:1088D000032811D1ECA10120FDF7A2FCECA1092095
:1088E000FDF79EFCDFF8B0C39CF80000F074FFF7C2
:1088F000FCF8F07C8CF8000096F82D00042811D1CB
:10890000E6A10120FDF78CFCE6A10920FDF788FC1B
:10891000E64B18787067FEF716FF96F8740018702B
:10892000C4E9028596F82D00052811D1E0A10120A7
:10893000FDF776FCE0A10920FDF772FCDFF880C3AB
:108940009CF80000F074FFF7D0F8F07C8CF8000081
:1089500096F82D00062813D1AFF2BC110120FDF7C7
:108960005FFCAFF678710920FDF75AFCDFF854C3BD
:108970009CF80000F074FFF7B8F8F07C8CF8000069
:1089800096F82D00072811D1CFA10120FDF748FC52
:10899000C2A10920FDF744FCDFF834C39CF80000B5
:1089A000F074FFF7A2F8F07C8CF8000096F82D0028
:1089B000082811D1C4A10120FDF732FCC5A109206E
:1089C000FDF72EFCDFF814C39CF80000F074FFF7ED
:1089D0008CF8F07C8CF8000096F82D00092818D14E
:1089E000B9A10120FDF71CFCBDA10920FDF718FC71
:1089F000707E012802D12168C9F80010D9F8000062
:108A00007067F0674FF47A704EF66021C4E9021087
:108A1000606096F82D000A2811D1B3A10120FDF75E
:108A2000FFFBA5A10920FDF7FBFBDFF8C4C29CF802
:108A30000000F074FFF759F8F07C8CF8000096F80D
:108A40002D000B2812D1AFF2BC210120FDF7E8FB6D
:108A50008FA10920FDF7E4FBDFF898C29CF8000025
:108A6000F074FFF742F8F07C8CF8000096F82D00C7
:108A70000C2811D1A0A10120FDF7D2FB89A109206A
:108A8000FDF7CEFB9E4B18787067FEF75CFE96F8FC
:108A9000740018700820A06096F82D000D2811D1E0
:108AA00098A10120FDF7BCFB98A10920FDF7B8FBB8
:108AB000DFF860C29CF80000F074FFF716F8F07C55
:108AC0008CF8000096F82D000E2812D1AFF2443138
:108AD0000120FDF7A5FB90A10920FDF7A1FBDFF820
:108AE00040C29CF80000F074FEF7FFFFF07C8CF8A9
:108AF000000096F82D0096F82E1088420FD189A11B
:108B00000120FDF78DFBAFF2D0210920FDF788FB96
:108B10004FF0FF3070676560707E012817D0834981
:108B20001120FDF77DFB716F002902DB1620FDF798
:108B300033FB706C401E70640BD0FEF758FA707EE9
:108B4000012810D002281BD003281DD001E086F890
:108B50002D7074A10120FDF763FBBDE8F047734958
:108B60000920FDF75DBBD4E901010A1AF16F8A42C1
:108B700001DAE06800E0084420608AF80070F5E55A
:108B8000E06820607776F8E796F82D0096F82E10CA
:108B9000884202D186F82D70E8E5401C86F82D0049
:108BA000E4E5634801F002BC10B5614C0020F03CE4
:108BB0005E4920720120FDF733FB5C490920FDF777
:108BC0002FFB0620216DFDF7E7FA207C012805D94F
:108BD000A16DBDE810400E20FDF7DEBA10BD2DE9F5
:108BE000F041534CF03C94F8370002283AD020462C
:108BF000E17AC078012601B110B9A17A002932D0FA
:108C0000207A38B1082001F06DFC092001F06AFCDF
:108C1000FFF7CAFF464DA07A0027703D78B1A772D2
:108C200002210020FDF712FC84F83760E8698047D4
:108C3000E07C40B14FF4FA6001F01EFA03E0A86A4C
:108C40008047E86A80473A488430007801F04AFC5F
:108C5000E772A07B00286DD1607C217C88426AD1BC
:108C6000207B69E003E1D8E020206C656674000099
:108C7000636F696E73000000BD0300202072696796
:108C800068740000BE0300202063687574650000EE
:108C90006D61746368000000BC030020637265644A
:108CA000697400006C696D6974000000D0030020D5
:108CB0002020636F696E0000736F756E647300002F
:108CC000CC030020C703002073706563696C00004B
:108CD000C20300206F76657272640000C103002039
:108CE00061776172640000002073636F7265000039
:108CF000CD030020C4030020657862616C6C000025
:108D0000D103002020204853544400006177617251
:108D100064200000C90300206164766E6365000072
:108D2000D40300206F7074696F6E0000DC79000856
:108D30004C0600205AE057E0FA490978884207D2E9
:108D4000401CC1B221730820FDF726FA66744DE07D
:108D500001210020FDF77AFB022084F83700F24859
:108D60000078A0B10A20A064FAF71BFB94F8481021
:108D70004843C1B2E1730820FDF70EFAE07B18B951
:108D800000210720FDF708FAFEF716FF04E0AFF216
:108D90000C610720FDF744FA206D28616067207C94
:108DA00001281AD0FEF7CAFE2969A06D0144296185
:108DB0006067207C022810D0FEF7C0FE2969206E73
:108DC000014429616067207C032806D0FEF7B6FEC7
:108DD0002969A06E014429616067FEF7AFFEFEF7C6
:108DE000E3FBF9F7DCFF01E0401C607494F8370006
:108DF000022832D0A8698047FDF7B6FBA07B38B1C6
:108E000004210120FDF722FBA07B401EA07301E09E
:108E1000FEF784FE286A80470CE078B9C348E67004
:108E2000007801F05FFBA07B4FF0040198B10120B6
:108E3000FDF70CFB94F8370002280ED04FF42F708A
:108E4000E06301F019F905210020FDF797FEBDE868
:108E5000F041FEF704B80020EAE7B54800780028A2
:108E600005D0BDE8F041B1480C3801F09FBABDE82B
:108E7000F081704770B50E460546012415E0295D66
:108E8000032905D9AB480078001F052802D202212A
:108E9000002000E00220FDF771FEA749305D09685F
:108EA000484301F0E9F8641CE4B22878A042E6D215
:108EB00070BDA04810B50078092813D903210020FF
:108EC000FDF75CFEFA2001F0D7F802210020FDF743
:108ED00055FEFA2001F0D0F80121BDE81040002035
:108EE000FDF74CBE9149BDE810409431A1F110004E
:108EF000C0E710B501210020FDF7A8FA8F480078DF
:108F0000FEF7ADFE894CFC3C04F82A0F8C48007833
:108F1000FEF7A5FE607085487C38C0698047002058
:108F2000A0722A3CFFF7C5FFFDF72BF900210620B0
:108F3000FDF732F97C48007850B10A20A064FAF7B6
:108F400030FAA16C48430146A0640820FDF724F9DB
:108F50007C48007820B17C4801781020FDF71CF98E
:108F6000607F28B194F8210080F0100084F821007F
:108F7000A07F20B114F8210F80F0200020706C48F1
:108F80000078002805D06948BDE810400C3801F091
:108F90000DBA10BD704710B56B4C207800280FD06B
:108FA000401E207067480078002809D0FF2110205B
:108FB000FDF7D0F82178BDE810401020FDF7ECB89F
:108FC00010BD70B5594C0026FC3C6048A664007882
:108FD00018B15D48007800287DD994F83700022840
:108FE00003D0607C01284CD06FE00A2001F07AFAAF
:108FF000032001F077FA042001F074FA062001F052
:1090000071FA072001F06EFAFDF7BBF8474D7C3D81
:1090100068698047A8698047082084F837000121E3
:10902000FDF7BAF8FFF7B7FF267503210020FDF71B
:109030000DFA04210020FDF709FA01210846FDF789
:1090400005FA02210020FDF701FAFFF700FB686A2C
:109050008047FDF789FA286A80474FF42F70E06354
:1090600001F00AF805210020FDF788FDFDF7F7FE65
:10907000374800686065E0656066E066FEF74EFDB3
:109080000BE0207C042820D2207B01281DD1294818
:109090000078102819D0FFF77EFF207C2D49401C56
:1090A000C0B220740A68521C0A60012818D0FFF769
:1090B000CEFA207C022816D003284FF0000115D0EC
:1090C0001E20BDE87040FDF767B8012084F831002C
:1090D00016486C3000E00BE0BDE8704001F066B966
:1090E00000210620EDE700210E20EAE71620E8E740
:1090F00070BD10B50D4CFC3C224694F8353092F80A
:109100003620012B28D0805C84F82200C1B294F86C
:109110003300FDF79BF994F83300F8B1002084F890
:10912000330010BDBB030020C403002058060020FC
:10913000CA0300202404002030040020BD030020C6
:10914000BE030020C7030020D2030020D00300206C
:10915000FC030020DC030020885CD5E70120DEE76B
:1091600070B500240D46224608E0295D04F1010493
:10917000E4B20029F9D102F10102D2B28242F4D361
:1091800004E0641CE4B20620FDF760F9295D0029C3
:10919000F7D170BD2DE9FF5F01241E469046814640
:1091A000A346FE4F254602EB060AFC747867444549
:1091B00004D8601EC0B20199FFF7D2FF282000F04A
:1091C0005BFFB9F1000F02D0786FFEF71DF9282080
:1091D00000F052FFB44205D9A01B401EC0B2019955
:1091E000FFF7BEFFA24502D10020F87408E0012C71
:1091F00003D0F87C20B1641C03E087F813B0FAE7D1
:10920000641E6D1CEDB2E4B2142DD0D9BDE8FF9FF1
:109210002DE9F047E14C01251E4617468846814658
:1092200084F83550FDF7CEF9DDA1E148FAF7FAFCF4
:10923000FEF74DFD4FF47A7000F01EFFFDF794F934
:10924000A56401210020FDF799FC02210120FDF712
:10925000FDF83C2000F010FF01210020FDF78EFCFE
:10926000FDF782F902210020FDF7F0F83C2000F024
:1092700003FFA06C401CA0640828E2D933463A469C
:1092800041464846FFF786FFFEF72CFD84F836502E
:10929000002084F83300C74801F088F8BDE8F047A3
:1092A000FDF79BB970B5BD4C94F8310001282BD166
:1092B000207A28B1082001F015F9092001F012F9EF
:1092C000A07A002520B1A57202210020FDF7BEF88A
:1092D0000E2001F007F9022001F004F9AF488030B8
:1092E000C0698047E07C18B14FF4FA6000F0C4FE1A
:1092F0000B2001F0F7F8E572A573022084F837001F
:10930000FFF75FFE84F8315070BDAB4810B50168BF
:10931000A24C491C0160A948007860B1A8480078B7
:10932000A06494F82A006067FEF76AFC94F8740061
:1093300084F82A000BE0A3480078A06494F82B007E
:109340006067FEF75DFC94F8740084F82B00A06C55
:1093500028B1FDF75CFFA06C401EA064F8E79A48B6
:109360000078002803D0BDE81040FEF782BCD8E6A4
:109370002DE9F041954801789548006831B195494B
:109380000978092902D3C0F3470600E0C6B2834D2D
:1093900091494FF47A77687BE0B36C7988461DE099
:1093A0006C710CE0FDF7D5FE3846FEF72DF830461F
:1093B00000F062FEFDF7F2FE6879401E6871687980
:1093C0000028EFD1D8F8000000F056FEA879012857
:1093D00002D9FEF74FF901E0401EA871A8790028D4
:1093E000DED144E5AC79FDF7B4FE07E03846FEF780
:1093F0000BF8304600F040FE641EE4B2002CF5D1BC
:10940000FDF7CCFE6879401E6871D8F8000000F0C6
:1094100033FE01E0FFE7884668790028E2D126E5BF
:10942000704770B55D4C002604F1D70184F83360B5
:10943000881FFFF71FFD694D2878E0742E7042F2F7
:1094400010706067FDF7E0FFE07C2870BDE87040B9
:10945000C82000F011BE624810B501684F4C491C8D
:109460000160022084F8370001210020FCF7EEFFA4
:1094700002210120FCF7EAFF4E48007801F032F8A3
:10948000E07840B90120E07004210020FCF7DEFF05
:10949000022001F027F8F9F782FC4E4800780A28EC
:1094A00017D24D4803210068E0630020FDF766FBFA
:1094B000E06B400000F0E0FD02210020FDF75EFBC4
:1094C000E06B00F0D9FD0121BDE810400020FDF760
:1094D00055BB26E610B5314CA07A00283AD194F855
:1094E0003700022836D03F480178A1B3607A0122C4
:1094F000401CC0B26072814237D1002060723A488D
:109500000168491C0160A27202210120FCF79EFF44
:10951000FA20E06303210020FDF730FBE06B00F050
:10952000ABFD03210020FDF729FBE06B00F0A4FD5B
:1095300003210020FDF722FBE06B00F09DFD0121DF
:109540000020FDF71BFB04F18000C06B8047042066
:1095500084F83700E5E5FFE7022084F837000121B1
:10956000BDE810400020FCF771BF2272082000F017
:10957000B9FF092000F0B6FF0E483C3800F016FF96
:109580000C48303800F012FF18A10120FCF748FE0B
:10959000BDE8104017A1092030E000005C05002064
:1095A000796F7520646177697A61726400000000E8
:1095B000470A0020D0060020E4030020BC0300205E
:1095C000BD030020BE030020CC030020C303002005
:1095D000280400202404002030040020CD030020B3
:1095E000EC030020D3030020F40300202077686FF1
:1095F000616800006275626261200000FCF710BEC5
:10960000A549487A002801D0401E48727047A249F7
:10961000002008757047A04890F8301019B100215B
:1096200080F830107047012180F830109A4880305F
:10963000006C0047984A10B5002302F180010F2802
:109640002DD2DFE800F02C080B0E112E1414171A7F
:109650001D1D1F222900FEF741F822E0FEF7B6F893
:109660001FE0FEF772FB1CE0FEF7A3FB19E0FEF71C
:1096700042FC16E0FFF7C4FF13E0FFF795FA10E095
:1096800013750EE0FFF7C7FF0BE00320FDF7B6FBF5
:1096900038B1FFF707FE04E0486C804701E0896CB1
:1096A000884700203DE5032811D005DC58B101288A
:1096B0000BD002280FD128E6042809D0052808D0AD
:1096C0000F2808D1C7E600F007BCFFF720B878E400
:1096D00000E7FFF784BA704770B5704800247249FC
:1096E00004706F48012504706E48047005200870EE
:1096F0006E4873A105706E4804606E4804606E4841
:1097000005706E4805707548FAF78CFA7448784908
:10971000032204707348944B0470734805707348B7
:10972000057040F6C41008607248754904707248AC
:10973000047072480860744972480860734875493B
:109740000460734808607448754905707348057073
:109750000F2008707348804905707348047073487F
:10976000027073480470734804607348046073485F
:10977000046073480460734804607348057073485C
:109780000460734805707348086075497348086041
:1097900074490C70C8211970744B1C70744B1D7087
:1097A000744D44F620632B60734B744D1C704FF462
:1097B0007A732B60724B1860734B72481860734851
:1097C00002707348734A047069201060724A106016
:1097D000724A10607248016070BD2DE9F0412E4C54
:1097E0000126002504F8136F6EA1C4F83550C4F8A3
:1097F0003950C4F86150C4F865506C48641CFAF7DD
:1098000011FA04F8095C25704FF00F0804F8148C65
:1098100066700A20A07004F8075C1F4FA566E5700B
:10982000803725713D606571A571022084F82300A1
:10983000E67125725BA107F15D007D60FAF7F2F930
:10984000A5626572A572E5722573FF206073A5732A
:1098500084F80F802420BD602074667484F813801F
:109860001020A074FD606575A675E67584F81880F3
:10987000667684F81A804EA107F16500FAF7D2F9EE
:109880003D614D48E57665770580A5774FF4167004
:109890002063E577A5E500005C050020B803002003
:1098A000B9030020BA030020BB030020BC03002042
:1098B000E0030020E4030020BD030020BE030020DD
:1098C00053797374656D3120435055202041524DBA
:1098D00020206D6F64656C2000000000D709002017
:1098E000BF030020C5030020C6030020C7030020DB
:1098F000D8030020C8030020D4030020C0D40100F6
:10990000FC0300207082030000040020DC03002020
:1099100000E2040004040020C9030020CA03002060
:10992000CF030020C4030020D0030020D103002077
:10993000D2030020E8030020EC030020F003002005
:1099400008040020F4030020CC0300200C040020B5
:10995000CD03002020BF020010040020C0450400F9
:1099600014040020CE030020C0030020C103002007
:10997000C203002018040020C3030020F8030020C5
:109980001C04002090D0030020040020D3030020FA
:10999000D50300202C0400203004002028040020DF
:1099A000340400206E756C6C00000000470A002033
:1099B000322E333700000000B403002010B5FDF74D
:1099C0007BFA032806D028B1FDF764FAFD49002090
:1099D000087010BD012010BD2DE9F041FA4FFB4D7C
:1099E0004FF49678C7F800802878F94E01240028B3
:1099F00068D0C0EBC00081190920C91FFCF710FC1A
:109A000023E0FDF799FA012804D002284AD0032860
:109A10001BD14BE0EB49002008702878062814D2AF
:109A2000DFE800F040030B0E111B24B10024204698
:109A3000FCF73AFC09E00124F9E7FCF7DEFD04E05D
:109A4000FDF7ECF801E0FDF7EBFA3868401E3860EE
:109A5000401CD6D10120BDE8F081FFF73DFEDD4876
:109A6000DD4A0068A0F59C4120391160DB4AA0F571
:109A7000EA4130391160DA49A0F51C4040380860ED
:109A80000120687003210020FDF778F8D5490920EE
:109A9000FCF7C6FB4FF4FA7000F0EEFACC491C312B
:109AA0000920ABE7FCF76DFB0020D4E7C7F8008086
:109AB000287801240621401CB0FBF1F201FB1200C2
:109AC000287094E7C749092098E72DE9F041BE4F77
:109AD0004FF49670C4A138600920FCF7A1FBC44C78
:109AE000DFF8E882207808F1020800EB800101EB42
:109AF000C00141441120FCF793FB267800252FE09C
:109B0000FDF71AFA012804D0022815D0032827D11E
:109B100015E0B848112105702078401CB0FBF1F227
:109B200001FB120000EB800101EBC00120704144F9
:109B30001120FCF775FB13E0257000208BE7AEA128
:109B40000920FCF76DFBACA11920FCF769FB20781C
:109B5000B04204D0F9F779F89C49012048703D6083
:109B60003868401E3860401CCAD1012073E72DE9D7
:109B7000F05FA34901240020DFF88892A24DDFF8AE
:109B80008C82A34EA34F08704FF0050A9AA10920BA
:109B9000FCF746FB012C10D0022C19D0032C2ED040
:109BA000042C40D0052C5AD0062C76D0072C71D02E
:109BB000082C70D0092C6FD0D4E097A10120FCF7BD
:109BC0002FFB97A10920FCF72BFBDFF85CB209E023
:109BD00096A10120FCF724FB91A10920FCF720FBB2
:109BE000DFF850B2DBF800002860D9F800008047A9
:109BF00029683220CBF800103860C8202AE08EA1F6
:109C00000120FCF70DFB8EA10920FCF709FBDFF812
:109C100038B29BF800002860D9F800008047287807
:109C20008BF8000012E084A10120FCF7F9FA7CA176
:109C30000920FCF7F5FADFF814B2DBF80000286021
:109C4000D9F8000080472968CBF8001064203860FC
:109C50004FF49670C8F80000C6F800A082E07CA11E
:109C60000120FCF7DDFA7CA10920FCF7D9FADFF826
:109C7000F0B19BF800002860D9F8000080472878F0
:109C80008BF800000A2038603220C8F8000001205C
:109C900038E002E01DE037E053E072A10120FCF75C
:109CA000BFFA72A10920FCF7BBFADFF8C8B1DBF8F4
:109CB00000002860D9F8000080472968CBF8001020
:109CC0004FF42F70386040F2DC516420C8F8001067
:109CD00018E064A10120FCF7A3FA67A10920FCF7B2
:109CE0009FFADFF89CB19BF800002860D9F80000CB
:109CF000804728788BF800001E20962138600A20C3
:109D0000C8F8001030602DE05EA10120FCF788FA51
:109D10005EA10920FCF784FA37A11120FCF780FA34
:109D2000DFF870B106E001210020FCF727FF3C209E
:109D300000F0A2F95848DBF8001000688142F2D028
:109D400010E056A10120FCF76BFA56A10920FCF7A0
:109D500067FA4FF0FF302860002030602848007814
:109D6000012818D024A11120FCF75AFA29680029EB
:109D700002DB1620FCF710FA13490868401E086041
:109D800009D0FDF734F91E49087801280DD00228C2
:109D900015D0032814D041A10120FCF741FABDE8F9
:109DA000F05F15A10920FCF73BBAD8F80010306825
:109DB0000A1A3E4909688A427ADA396879E07CE011
:109DC00083E075E040080020440800204807002098
:109DD000A902002004040020140400202004002014
:109DE000000400207802002073656C656374000035
:109DF00024040020B8030020202020202020000080
:109E00007505002070040020D0050020E405002026
:109E1000E0050020E80500202073636F72650000F4
:109E20006C616720746D00003004002020626F6E4A
:109E300075730000280400202020636F696C000007
:109E4000686C6420746D0000C0030020340400209E
:109E500020206C616D700000656E6120746D0000E3
:109E6000CF030020737769746368000073747220F5
:109E7000746D0000F803002064757020746D00009C
:109E800008070020202054696D65000063616C693B
:109E9000627200004C050020500500206578706556
:109EA00072740000646F6E6520200000D8050020E9
:109EB000014458480160012004E056483A680260B5
:109EC000012008705449487060E6092C02D0641CD7
:109ED000E4B25BE6012459E62DE9F047FCF751F9BD
:109EE000DFF8349101214D4E89F800100D464FF0F6
:109EF000000A4FF4167889F801A04446F11D44E0A9
:109F0000FDF71AF8012804D002282DD003283FD1EC
:109F10002CE0C5EBC50081190F460120FCF780F944
:109F2000072D16D2DFE805F02004070A0D101300F4
:109F3000FEF745F90DE0FDF770FC0AE0FFF74CFD78
:109F400007E0FEF705FC04E0FFF7BFFD01E0FFF7C7
:109F50000EFE002C08DD444639460120FCF760F96E
:109F6000AFF26C11112011E0002411E02C486D1C9F
:109F700044460078EDB208B1072000E00620A84270
:109F800000D10025C5EBC50081190120FCF748F977
:109F9000201EA4F10104B3DC99F801004C4658B12D
:109FA00020A10120FCF73CF920A10920FCF738F999
:109FB000F8F7F5FE84F801A04FF4487000F05CF863
:109FC0001C4902200870FCF7DCF81B48007828B117
:109FD0001A4801781020FCF7DFF804E0AFF2E41132
:109FE0000F20FCF71DF916480178BDE8F04708205E
:109FF000FCF7D2B8134810B50168491C0160012173
:10A000000020FCF723FAF8F7CAFEBDE81040F6F787
:10A010009EBB0000DC0500204807002078020020DD
:10A02000D4030020736176696E6700006E767261FA
:10A030006D20000093050020C7030020D2030020FC
:10A04000C4030020EC03002010B502460020F74CAA
:10A05000207001210CE0012305E0F448007808B1EC
:10A06000084610BD5B1C40F6A6608342F5D9491C2A
:10A070009142F0D90020F4E710B501210CE0012253
:10A0800005E0EA4C24780CB140F6A663521C40F679
:10A09000A664A242F5D9491C8142F0D910BD002026
:10A0A000E3490880E3490870E3490870E349087010
:10A0B00040F26D10E24908800420E24908707047C0
:10A0C000E0480078E04908700520DE4908707047D4
:10A0D000DD480078DB49087070474188D44A118018
:10A0E0008179D44A11704179D34A11700179D34AE8
:10A0F00011700188D24A1180D44AC16811600321CD
:10A10000D04A11707047D2480088D2490880D2489E
:10A1100000780871D14800784871D148007888717A
:10A12000D04800884880704700B50346FFF7EBFF32
:10A13000C84840881844801F82B24FF47A7092FB5E
:10A14000F0F100FB1120C34948804FF47A7092FB74
:10A15000F0F082B2002A34DD08468079104482B2E1
:10A160003C2092FBF0F100FB1120BA4988713C20A1
:10A1700092FBF0F082B2002A23DD084640791044B9
:10A1800082B23C2092FBF0F100FB1120B1494871F2
:10A190003C2092FBF0F082B2002A12DD08460079E2
:10A1A000104482B2182092FBF0F100FB1120A94963
:10A1B0000871182092FBF0F082B208460088104423
:10A1C000088000BD9E480088A24908809B4800780E
:10A1D00008719948007848719648007888719448C9
:10A1E000008848807047002008E0002100EB400212
:10A1F0009D4B03EBC2021172411CC8B22028F4DB54
:10A2000000219A4A11607047024602B111B96FF0FD
:10A210000200704710880B88984201DD0120F8E7A2
:10A2200010880B88984202DA4FF0FF30F1E710797E
:10A230000B79984201DD0120EBE710790B79984208
:10A2400002DA4FF0FF30E4E750794B79984201DDB4
:10A250000120DEE750794B79984202DA4FF0FF3067
:10A26000D7E790798B79984201DD0120D1E7907989
:10A270008B79984202DA4FF0FF30CAE750884B885A
:10A28000984201DD0120C4E750884B88984202DAE9
:10A290004FF0FF30BDE70020BBE730B50246108825
:10A2A0000D88431B1BB1002B00DA22E040E010793F
:10A2B0000D79441B1CB1002C00DA21E03FE05079FD
:10A2C0004D79431B1BB1002B00DA20E03EE0907972
:10A2D0008D79441B1CB1002C00DA1FE03DE0508852
:10A2E0004D88431B002B02DA584200B230BD18B231
:10A2F000FCE708791579401B182505FB030400BF0E
:10A3000048795579401B3C2505FB040300BF88793B
:10A310009579401B3C2505FB030400BF4888558800
:10A32000401B4FF47A7505FB0403584200B2DDE789
:10A3300010790D79401B182505FB030400BF5079E7
:10A340004D79401B3C2505FB040300BF90798D79B6
:10A35000401B3C2505FB030400BF50884D88401B73
:10A360004FF47A7505FB040318B2BFE770B50446D5
:10A370003E48056801E02E466D6929462046FFF7F4
:10A3800043FF0028F7DC39480068854202D037488F
:10A39000006840B93548006860613448046000686E
:10A3A000FFF79BFE01E07461656170BD70B5044606
:10A3B000A088642802DA6FF0010070BD002601E079
:10A3C000701CC6B2202E07DA06EB4600264901EBC8
:10A3D000C000007A0028F3D1202E02D14FF0FF30C8
:10A3E000EBE706EB4600204901EBC005A088FFF72C
:10A3F0009BFE1848016829608188A9808079A8712E
:10A40000A088288260786872A078E8712078287225
:10A41000A068E8602846FFF7A9FF0020CDE710B547
:10A420001248006808B900244CE021E040080020F0
:10A430002E08002037080020390800203B080020A3
:10A4400034080020B20300205008002054080020E7
:10A4500032080020D80D00203A08002038080020DB
:10A46000360800202C080020D80A002048080020C8
:10A470003448046834480078022803D1607AFFF732
:10A48000D9F801E0E06880472E48006840692D490E
:10A490000860E079012802D10020207212E0E07902
:10A4A000002802DDE079401EE071208AFFF73CFEC3
:10A4B0002648016821608188A1808079A0712046AA
:10A4C000FFF754FF1F48006818B904201E490870A0
:10A4D00007E01C480068A04203D01A480068FFF754
:10A4E000FCFD10BD30B505461648006810B94FF0A8
:10A4F000FF3030BD1348036801E01C465B6913B1AF
:10A50000187AA842F9D113B94FF0FF30F1E70D489E
:10A510000068984206D106200B490870094958691D
:10A52000086001E058696061002018720548006801
:10A5300020B104480068FFF7D0FD01E0FFF7AFFD50
:10A540000020D6E748080020B2030020D80D0020E4
:0CA5500001000000960000008D6600086D
